:1000000000308A00D22D0000FF00030E8301A10002
:100010007F08A0000A08A8008A01A00E0408A20018
:100020007708A3007808A4007908A5007A08A6003C
:100030007B08A700831383128C308400001C2228C5
:100040000C184628220884002308F7002408F8002A
:100050002508F9002608FA002708FB0028088A006E
:10006000210E8300FF0E7F0E09000A108A100A116C
:1000700082070334F33425346134D13449340934EC
:10008000E33401344134FF343D34FD34B90A0030E7
:10009000AD02031C0130AE020130031C0230AF027E
:1000A0000030031C0130B002B008031D6A282F087D
:1000B000003C031C6A283108AD0732080318320FD0
:1000C000AE0733080318330FAF0734080318340F93
:1000D000B007B50A0310340CFA00330CF900320CE7
:1000E000F800310CF70030087A02031C8B28031D3E
:1000F00089282F087902031C8B28031D89282E08C4
:100100007802031C8B28031D892877082D02031809
:100110008B28B6018D280130B60035083C3C031D04
:10012000D528C20AB50142083C3C031DD528C10AA6
:10013000C2014108183C031DD528C00AC10140086E
:100140001D3C031DAB283F08023C031DAB283E08A5
:100150000339031DCB2840081E3C031DB3283F086C
:10016000023C0319CB2840081F3C031DC7283F0849
:10017000043C0319CB283F08063C0319CB283F0851
:10018000093C0319CB283F080B3C0319CB28400836
:10019000203C031DCE28BF0A0130C0003F080D3CA3
:1001A000031DD528BE0A0130BF000C108A11222879
:1001B00054308400831300080319EC280130F80040
:1001C000F701F70BE128F80BE0284A30F700F70BAE
:1001D000E728EA28800BDE280034D30152085302B6
:1001E000031834298316860183124E08860083166D
:1001F0000510831205140330D400D820831605108F
:10020000831205108316860183124F088600831619
:100210008510831285140330D400D82083168510EE
:100220008312851083168601831250088600831678
:100230000511831205150330D400D820831605114B
:1002400083120511831686018312510886008316D6
:100250008511831285150330D400D82083168511AB
:1002600083128511D30AEE28831686018312860134
:1002700000343408B0003308AF003208AE00310853
:10028000AD008530900083160C148312192E4F0890
:10029000F8014E0203184F294E08F7005B29F701B9
:1002A0000830D000CE0DF70D4F0877020318F70085
:1002B000F80DD00B52290034D2015208093C031C1E
:1002C000A9298316860183124E088600831605101D
:1002D000831205140330D400D8208316051083122E
:1002E00005108316860183124F0886008316851039
:1002F000831285140330D400D8208316851083120E
:10030000851050083520D3008316860183125308C8
:10031000860083160511831205150330D400D820FA
:10032000831605118312051151083520D300831659
:100330008601831253088600831685118312851562
:100340000330D400D8208316851183128511D20A78
:100350005D298316860183128601003483160614F4
:100360008312061CBD290230CE009630D400D8205E
:10037000CE0BB5290130F800D929831686148312D3
:10038000861CD0293130CE003930CF00B930D000B2
:100390000D30D1005030D200ED200230F800D929C4
:1003A0000230CE009630D400D820CE0BD2290030B7
:1003B000F8000034831606148312061C292AB80A92
:1003C0000230CA009630D400D820CA0BE22938087F
:1003D000033C031CB80138080319F829013A031932
:1003E000042A033A0319102A013A03191C2A282A5D
:1003F0009130CE003930CF003B30D000BD30D1003D
:100400005030D200ED20292A3130CE008130CF008B
:100410001D30D0000D30D1005030D200ED20292AFF
:100420004930CE000D30CF000F30D000FF30D1006A
:100430005030D200ED20292A1D30CE009130CF005F
:100440000D30D000BD30D1005030D200ED20292A2F
:10045000292A831686148312861C5A2C9130CE00CA
:100460003930CF009F30D0003130D1005030D20031
:10047000ED20B801831686148312861C5A2C49304D
:10048000CE000D30CF001D30D000FF30D1005030F5
:10049000D200ED20CC014D104D18742A3E08CE003C
:1004A0000A30CF0047217808CA003E08CE000A3043
:1004B000CF0047217708CB005130CE00BD30CF00B0
:1004C0004A08D0004B08D1005C21AE217808CC004E
:1004D0004C0B6F2ABE0A3E08643C0319BE014C084F
:1004E000023C03194D144C2ACC014D104D18A02A82
:1004F0003F08CE000A30CF0047217808CA003F08E5
:10050000CE000A30CF0047217708CB008730CE00DD
:10051000C330CF004A08D0004B08D1005C21AE2187
:100520007808CC004C0B9B2ABF0A3F080D3C031DEA
:100530009B2A0130BF004C08023C03194D14762A57
:10054000CC014D104D18F42A4008CE000A30CF00DF
:1005500047217808CB004008CE000A30CF00472161
:100560007708CC003130CE005130CF004B08D0009E
:100570004C08D1005C21AE217808CA004A0BEF2A52
:10058000C00A40081D3C031DCD2A3F08023C031D44
:10059000CD2A3E080339031DED2A40081E3C031DE9
:1005A000D52A3F08023C0319ED2A40081F3C031DD1
:1005B000E92A3F08043C0319ED2A3F08063C0319C9
:1005C000ED2A3F08093C0319ED2A3F080B3C0319AB
:1005D000ED2A4008203C031DEF2A0130C0004A08E4
:1005E000023C03194D14A22ACC014D104D181E2BAC
:1005F0004108CE000A30CF0047217808CA004108E0
:10060000CE000A30CF0047217708CB009130CE00D2
:10061000BD30CF004A08D0004B08D1005C21AE218C
:100620007808CC004C0B192BC10A4108173C031C5D
:10063000C1014C08023C03194D14F62ACC014D109F
:100640004D18472B4208CE000A30CF0047217808CA
:10065000CA004208CE000A30CF0047217708CB00FD
:10066000B930CE00CF004A08D0004B08D1005C2141
:10067000AE217808CC004C0B422BC20A42083B3C0E
:10068000031CC2014C08023C03194D14202BCC0161
:100690004D104D18702B3508CE000A30CF00472181
:1006A0007808CA003508CE000A30CF004721770805
:1006B000CB00FF30CE00CF004A08D0004B08D1005D
:1006C0005C21AE217808CC004C0B6B2B35081D3C0F
:1006D000031CC20AB5014C08023C03194D14492BF6
:1006E000CC014D10013083169B009C131C141A087A
:1006F0008312AC01AB01AA01A9002908CB0031305B
:10070000CE00BD30CF008D30D0001D30D100503034
:10071000D200ED204D18182C0A30BA004B08CE003C
:100720000A30CF0047217708BD004B08CE000A30C1
:10073000CF0047217808CB004B08CE000A30CF000D
:1007400047217708BC004B08CE000A30CF00472174
:100750007808BB00CA014A08183C031C012C3A085F
:100760003520CE008316860183124E08860083163C
:100770000510831205140330D400D8208316051009
:10078000831205103B083520CE00831686018312A4
:100790004E08860083168510831285140330D4001A
:1007A000D82083168510831285103C083520CE0092
:1007B0008316860183124E08860083160511831264
:1007C00005150330D400D8208316051183120511B6
:1007D0003D083520CE008316860183124E08860020
:1007E00083168511831285150330D400D820831613
:1007F0008511831285118316860183128601CA0A28
:10080000AB2BAE217808CC004C0B112C0130A90782
:100810000318AA0A0319AB0A0319AC0A4B0F112CCF
:10082000CB014C08023C03194D142908CB008A2B3C
:10083000013083169B009C131C141A088312CB00F2
:1008400029084B02031D2D2CAA08031D2D2CAB08D3
:10085000031D2D2CAC080319452C013083169B0079
:100860008312290883169A001C1583120B08F700BF
:100870008B13831655309D00AA309D009C149C1844
:100880003F2C1C11770883128B0440302907B100DC
:100890002A08B200423003184330B2072B08B300D5
:1008A0000F3003181030B3072C08B40000300318C1
:1008B0000130B4073A083520CA0083168601831236
:1008C0004A08860083160510831205140330D400ED
:1008D000D82083160510831205103B083520CA0066
:1008E0008316860183124A088600831685108312B8
:1008F00085140330D400D820831685108312851008
:100900003C0835203706CB008316860183124B083E
:10091000860083160511831205150330D400D820F4
:1009200083160511831205113D083520CA00831670
:10093000860183124A088600831685118312851565
:100940000330D400D82083168511831285118316B5
:100950008601831286010034CA014A08073C031C41
:10096000CC2C8316051283120512B62C831605169D
:100970000230F700F70BBA2C000005168312051A97
:10098000C32C0310C42C0314CB0C2730F700F70B37
:10099000C72CCA2CCA0AAD2C4B08F80000348316A9
:1009A000051283120512A630F700F70BD52C0000B4
:1009B00083160516A630F700F70BDC2C0000051691
:1009C00083120034CB014B08073C031CFF2C831619
:1009D000051283120512EC2C0310CA0C0318F22C1A
:1009E0000512F32C0516831605121330F700F70BCA
:1009F000F72CFA2C0516FC2C8312CB0AE32C0034BE
:100A0000C301C601C308031D0E2D3808033C031D96
:100A10000E2DAC247808C300DA21022DCF24CC306F
:100A2000CA00E224BE30CA00E224AC247808C40024
:100A3000AC247808C500AC247808C700AC2478083A
:100A4000C800AC247808C900AC247808C900AC24DC
:100A50007808C900DA210130B7000310C40C490836
:100A60001C3CC60046080F3C0318392D1030C60246
:100A70003A2DC4034608CA000A30CB00F701F8013A
:100A80004A0803104B18F707F70CF80CCB18F707B8
:100A9000F70CF80C4B19F707F70CF80CCB19F70704
:100AA000F70CF80C4B1AF707F70CF80CCB1AF707F2
:100AB000F70CF80C4B1BF707F70CF80CCB1BF707E0
:100AC000F70CF80C7808C600C60E0F30C605450FA7
:100AD000752D0C30BA007F30C406C6080319742D7A
:100AE00046080A3CC600752DC40A4408633C031836
:100AF000882D4408CE000A30CF0047217708C60071
:100B00004408CE000A30CF0047217808C400B7015E
:100B1000450F9D2D4408093C03189D2D4408CE0027
:100B20000A30CF0047217708C6004408CE000A30BB
:100B3000CF0047217808C400B7010B30BD0046083C
:100B4000BC004408CE000A30CF0047217708BB0024
:100B5000450FAD2D0C30BA00BB2D4408093C0318DD
:100B6000B92D4408CE000A30CF0047217808BA00DA
:100B7000BB2D0A30BA00DA210310350CCB00CE00B1
:100B80000630CF004721770BCA2DB808031DCA2DA8
:100B9000DA21BC2DCF24CC30CA00E2244430CA0074
:100BA000E2240034840183131F30830507309F0043
:100BB0006430A900AA01AB01AC01B501B601B701CF
:100BC0000330B800B901BA01BB01BC01BD01BE01CF
:100BD0000130BF00C000C101C2013F3065000030DC
:100BE0006600CE01CF01D001D101FF30D200ED204F
:100BF000013083169B009C131C141A088312AC014D
:100C0000AB01AA01A90040302907B1002A08B200AF
:100C1000423003184330B2072B08B3000F300318DB
:100C20001030B3072C08B400003003180130B407AB
:100C30003929C0308B04B808031D812E0310350CF0
:100C4000C500CE000630CF004721F708031D522E05
:100C50000130B7004008CE000A30CF0047217808A5
:100C6000BA00BA08031D362E0A30BA004008CE007A
:100C70000A30CF0047217708BB003F08CE000A307A
:100C8000CF0047217808BC00BC08031D492E0A305C
:100C9000BC003F08CE000A30CF0047217708BD00D6
:100CA000DA21812E0310350CC400CE000630CF00AF
:100CB0004721770B5D2E0025812E3608B7004108AD
:100CC000CE000A30CF0047217808BA004108CE0094
:100CD0000A30CF0047217708BB004208CE000A3017
:100CE000CF0047217808BC004208CE000A30CF0070
:100CF00047217708BD00BA08031D802E0A30BA00CC
:100D0000DA21380BAC2E0130B7004008CE000A3093
:100D1000CF0047217808BA00BA08031D912E0A3087
:100D2000BA004008CE000A30CF0047217708BB0048
:100D30003F08CE000A30CF0047217808BC00BC082D
:100D4000031DA42E0A30BC003F08CE000A30CF009D
:100D500047217708BD00DA213808023C031DCF2E59
:100D60003608B7004208CE000A30CF004721780885
:100D7000BA004208CE000A30CF0047217708BB00F6
:100D80003508CE000A30CF0047217808BC0035086E
:100D9000CE000A30CF0047217708BD00DA2138089D
:0A0DA000033C031900251B2E63001D
:02400E00013F70
:00000001FF
